S01B000070705F476E6F6D5F31335F4176746F4E756C2B70756C7365D5
S1130000F4C018951895189518951895189518957D
S1130010189518950150104098018901232BD1F7A8
S1130020089510E01FBB0EBBE09A0DB30895202F76
S113003030E03FBB2EBB1DBBE29AE19AE199FECFB3
S1130040089512E813BF06BF00E21EE4E3DF00E0F8
S113005003BF089515D1C350B99ABC9A02EE06B9EC
S113006003E007B900E21EE4D5DF02E50FBD00E8B6
S113007008B9C49A00E2E5DF00E4E3DF00E8E1DF69
S113008000E41FE1C7DF00E2DCDFC49800E003BF47
S11300900AE0C7DF0395102F0AE0C9DF08EE1DEF61
S11300A0B9DF6624772488249924AA24BB24DD2478
S11300B012C015B100E024B130E0022B132B212F24
S11300C0220F220B322F800E911EA21EB31E04E1BA
S11300D010E0A0DFD39400E4D01658F388159905F6
S11300E0AA05BB052CF48F5F9F4FAF4FBF4F04C0D1
S11300F081509040A040B0400881002321F4C40105
S1130100D50107E008838C019D01081919092A0902
S11301103B09053640E0140740E0240740E034077B
S1130120BCF1C49AE3944E2DE42E442311F440E030
S1130130488341E0440E40E0541E49825A8249807B
S11301405A804CE050E060E070E04A015B0148EE08
S113015053E060E070E073D0801A910AA20AB30AF7
S113016009811A8120E030E080169106A206B306C8
S1130170E4F444245524CC24F0940FEFF01629F42D
S113018002E803BF04E206BF10C000E003BF0DC0D5
S113019000E003BFC49800E0F02EE02EC3940C2DC1
S11301A0C02E002311F400E0088301E0600E00E09B
S11301B0701E8301380101322EE4120708F473CF54
S11301C066247724DD2403E0D01608F06CCFC49AAB
S11301D004E237DFC49800E41CE91CDF00E0088374
S11301E0D394F1CF00008895FECF0FE90DBFC0E88E
S11301F058D030DFF7DFF6CF002411241001E0E2FD
S1130200EA9592F0001F111F221F331F001C111CBE
S1130210221C331C041615062606370688F3041A16
S1130220150A260A370AECCF001F111F221F331F9D
S1130230A001B10100951095209530950895FF27F0
S1130240772312F4F16014D0332312F4F09508D01C
S1130250D3DFF69508F404D0F69508F409C00895A0
S113026030952095109501951F4F2F4F3F4F0895BE
S113027070956095509541955F4F6F4F7F4F0895EE
S1130280FA92EA92DA92CA92BA92AA929A928A92CA
S11302907A926A925A924A92BA93AA939A938A93B6
S10902A0089501E0089539
S9030000FC
